:10740000E0E0F0E0859194910196089520E82093C2
:1074100061001092610081E085BF82E085BF81EF4D
:1074200085B987EE84B91DB8769A10BA80EF81BB12
:1074300084E68BB984EF8AB980E58CBD81E08DBD8F
:10744000089580EE8BB98BEA5AD0109289008AEFAA
:107450008093880082E080936F0083E080938100B6
:107460006CD06BD05C98E7E0F1E05ED0EA31E9F7F0
:10747000ADEEB3E0EAE1F1E003E010E101900D923E
:107480001A95E1F7A059BF4F0A95B9F756D081E098
:107490008093D7008AE482BF1092D8001092E20055
:1074A0001092DA001092E10080E808D019BC1EBAF0
:1074B0001092E0006DD489E059D481E98093D8001E
:1074C0000895F201F999FECFF2BDE1BD0895F9DF0B
:1074D000F89A80B508C0F5DF1FBA80BD0FB6F894E2
:1074E000FA9AF99A0FBE31962F010895A5EBB1E0F3
:1074F00090E81BD08D939A95E1F7089586E008D027
:1075000010C083E005D08F2F10D08E2F0ED080E0DA
:107510005E9A5A980AC005D085E0FADF06D080FD51
:10752000FDCF5A9A5E98089581918EBD8DB5000069
:1075300087FFFCCF8EB50895F4DFE5ECF2E05C9AAE
:1075400040E358E06081718198E08FEF60FF8F70B9
:1075500070FF807FEADF669576959A95B1F7E058DF
:10756000FF4F5A9579F7EE5FF3404A9551F708952A
:10757000E3EAF1E081919081019690838293092E54
:107580000AF400940091A10106FB5EF0009692912E
:1075900011F493959083000C081620F42E9A2F9ADC
:1075A0002D9A0895937009F42E98913009F42F982C
:1075B000923009F42D980895EAE9F1E09781992332
:1075C000EAF08FB18095807F669B88601C9B846009
:1075D0009581891310C09681992381F49381891331
:1075E00006C09481992396E959F080E00AC083830C
:1075F0009095892304C085839AE0968380E09FEF6D
:107600009483828308958091A10186FFC7DF22249D
:107610003324E5EBF1E080919C0187FD36C084FDC9
:107620004DC082FF089526842220E1F3F894C0899A
:10763000D78520E030E080E090E4AFEFBFEF119617
:1076400082199040E0F72D01BB4A8D0127FD13C040
:10765000E2E5F4E011928EE7819392E4E1179193D1
:107660009AE508F092E4E539C9F78193108264DF66
:10767000FE01219646DF3ADFF9011CD320583F4F27
:10768000040D151D2A9411F7A6C18301282D6090C1
:10769000BE017090BD0146D019F48823C1F708954A
:1076A000380188243FD0E1F58091BC01821709F4AC
:1076B00083016090C0017090BF01F4CF6090C00161
:1076C0007090BF012FD081F48823C1F708959FEFF8
:1076D00085FD08C086FD05C083FF089591DEE9F3AE
:1076E0007AC191E097FB890E6624772483012227D3
:1076F00019D0B1F4882389F38091BC0136F0881643
:1077000050F4821730F0213003C0881520F4281778
:1077100010F48301282F6090C0017090BF01E8CF62
:107720003801822EF301EDDEE1DEC5EBD1E0E0E0D1
:10773000F1E097E009908191081621F49A95D1F72C
:1077400008808010EECEC9E0D3DECA95E9F7F4DEFA
:0477500088270895E9
:1077540041524455424F5915103F75306FA055A101
:1077640000A200A87F81CFB121AF0000FFFFCFCFDF
:10777400FFFFFFFFCFCFFFFF0000FE067E7E06FE69
:1077840046565616FE0656461EFE3F61E9E3FFE3E3
:10779400EBE3FFE3EBE3FFE16B3F120110010200B7
:1077A40000084123360001000000000109023E00E8
:1077B40002010080320904000001020201000524D4
:1077C40000100104240204052406000107058203B5
:1077D4000800FF09040100020A0000000705040272
:0A77E40010000107058302100001E8
:1078000011241FBE8DEF9AE09EBF8DBF04B714BE3A
:1078100088E18093600010926000409100085091D0
:1078200001086F917F91A6C00F928F939F931F9233
:107830000FB60F9211244F936F938091DA0080FF5F
:107840004CC038C00F920FB68F939F93EF93FF9366
:1078500088278093850080938400EAE9F1E097818E
:10786000907261F490818917980B908309F45D9A66
:1078700091818917980B918309F4289A96819150E8
:1078800008F096839481915008F09483881639F417
:107890007C9B05C0B5DD19F0C10101961C01FF916B
:1078A000EF915CC080E189BD82E189BD09B400FE31
:1078B000FDCF08958091D80080FF0FC08091DA003D
:1078C0008E7F8093DA008091D90080FF04C0EADFC8
:1078D00081E08EBB02C019BC1EBA8091E10080FF1E
:1078E0000BC03ED280FF08C03ED28091D80080629B
:1078F000E5DD19BC85E08EBB8091E10084FF1AC0F4
:107900002FD284FF17C0CEDF8091D8008F7DD6DDC7
:107910008FEE2AD025D28F7E816028D28091A5015A
:10792000882331F48091E30087FD02C081E001C02B
:1079300084E08EBB8091E10083FF0CC011D283FFF5
:1079400009C087EF11D082E08EBB1092A5010BD049
:107950000AD21ED26F914F910F901F909F918F91DD
:107960000FBE0F9018958EEF0090E1000822009254
:10797000E10008954BDDA0E0B1E0E4E5F7E7059014
:107980000D92AA39E1F71D92BB30E9F701FD0FC056
:1079900000FF03C07C9B0BC008C003FF08C06757F3
:1079A000774729F04757574711F02ADDA1F449DD01
:1079B0002224332431018824B5DE789447D0FDD2C7
:1079C000FBDD85DE811411F01EDEF8CFD1DDC101B3
:1079D000805B964398F3F89489EB91DD81E0809386
:1079E000E00010926F0010928100109285001092BA
:1079F000840081E085BF15BED1DD5D9A289A0C9484
:107A00000000A9D107C054D102C0D4D239F0A5D109
:107A100082FFFBCF85FFF7CF8091F1000895082EFC
:107A200083E09AD185FD07C08FD102C0C3D269F02F
:107A300094D180FFFBCF0092F1008091A10185FBE2
:107A400026F05D9884E680939A01089584D182FFA0
:107A50004CC18091A10185FB26F0289884E6809393
:107A60009B01CFDF182F853431F48CEB94E31C019C
:107A700028DD8DE008C1843511F4C3DFFACF8C34E2
:107A8000C1F38035B1F3843721F484E4C8DF80E0AA
:107A9000FAC0813611F489E5F6C0813429F4B1DFEA
:107AA000582EAFDF482EE5CF803711F483E5EBC0C9
:107AB000833539F4C0E0D1E08991B1DFC730E1F717
:107AC000E3C0863521F481E3AADF84E3DCC0863796
:107AD00061F481E3669B8E5F1C9B8F5FA0DF8FB19B
:107AE000809582958F708F5BCEC08837A9F489DF2F
:107AF0008093A101289A84FD28985D9A83FD5D9862
:107B00002E9A81FD2E982F9A82FD2F982D9A80FD16
:107B10002D9887FD8824ADCF8A3649F48FE9F8DCAB
:107B2000C3E003DD7CDFCA95E1F7FBDCADC0833742
:107B300031F487E874DF85E972DF8EE1A4C0853611
:107B400039F4E0E8F3E7C9D0E058F040E0F791CF2E
:107B5000823631F489E563DF80E061DF80E893C03D
:107B6000823419F0873609F07AC02224332449DFA1
:107B7000D82F47DFC82F45DF082F8354843008F003
:107B800081C0063411F4440C551CF20110926F00B0
:107B90001736A1F4033471F483E0B4DCC6DC3FDFB4
:107BA0002197E1F7BEDC08C0063411F4859101C0CD
:107BB0008EDC35DF2197C2F72F0149C00334A1F4D1
:107BC0008E2F8F7021F49ADC80E29CDCA4DC96DCA2
:107BD00082E098DC16DFA9DCCA95E1F79CDC3196DF
:107BE000DA9571F72F0131C00634F1F49F01F437B3
:107BF000D8F473D019C005DF063461F4C0FB46F039
:107C0000F43728F4182E81E087BFE89511243296C6
:107C1000082E0AC0043439F4DF01B370AB54BD4FF1
:107C20008D93319601C057DC21972AF7043431F443
:107C30002F01F370FE2B49F480DC07C0063429F4D1
:107C40002F01F901F43708F446D08DE0E8DE063460
:107C500011F45694479482E080936F0015C08237E8
:107C6000E1E049F08634E0E031F08E34E3E019F0F1
:107C7000813531F4E2E0F0E089E087BF849103C010
:107C80008B3111F08FE3CBDE83E0A4D15DD095FF83
:107C900003C009C08FD149F160D080FFFBCF54D021
:107CA00002C088D111F159D080FFFBCF84E092D17E
:107CB0008BE74BC0A5EBB1E0F437B8F40ED090E4FD
:107CC0000D901D9081E087BFE89532969A95C1F797
:107CD0001124E058F04085E001C083E001D081E14B
:107CE00087BFE89507B600FCFDCF08959091AD01E0
:107CF0008091AE01913231F0913A61F5813251F5C6
:107D000038D078C0803231F534D054D1E9F08530A4
:107D1000D9F023D083FD18C082FFF7CF04C07CDEEA
:107D20008193615031F09091F3008091F200892BA2
:107D3000B1F7BEDF611549F704C03CD129F08530A9
:107D400019F00BD080FFF9CF8EE79091E8008923DE
:107D50008093E800089584E03DD18091E800089583
:107D60008091E2000895FCDF8E7F80618093E200C5
:107D700008951ED1E6EAF1E067E0089582E061EC43
:107D800009D083E061E802D084E060E842E103C00A
:107D900080E060E042E01ED181E007D01092ED006B
:107DA0006093EC004093ED0008959091EB00892BD7
:107DB0008093EB00089560E0923029F0913031F427
:107DC000EAE462E103C0ECE56EE300C0F1E008958F
:107DD0008091AD0188234CF402C0ECD051F0BDDF9E
:107DE00082FFFBCF65CFE6D021F0B7DF80FFFBCF6E
:107DF000ABDF08954091B3015091B401461751058E
:107E000010F490E028C0611511F0462FFACF9CDFE6
:107E100040E0F7CFCFD059F1853049F19EDF83FDA7
:107E200047CF9BDF82FD20C080FF15C03091F3005B
:107E30002091F20005C081918093F10041502F5FA5
:107E4000411519F028303105B0F350E028303105E4
:107E500009F451E079DF4115E9F65523D9F604C05C
:107E6000A9D029F0853019F078DF82FFF9CF20CF33
:107E7000EDEAF1E0D1DD8193E53BE1F737DF6DDF3E
:107E800083FF91C08091AD019091AE01913009F1D5
:107E900070F09330F1F0953009F444C0963009F455
:107EA00056C0983009F460C0993059F767C08238DD
:107EB00041F78091B1018DD02091EB001092E90043
:107EC00077D02295269521702093F1001092F10031
:107ED00052C0882311F08230A1F68F71823089F66A
:107EE0008091AF018823D1F42091B101277049F22C
:107EF0002093E9008091EB0080FF10C0933011F4D3
:107F000080E20BC080E151DF81E0880F2A95E9F71C
:107F10008093EA001092EA0088E047DF1092E900BF
:107F200047D02AC0882391F41091AF0110680FB791
:107F3000F8943ED04DDF11DF80FFFDCF1093E300BA
:107F4000103883E009F482E08EBB0FBF2CC080584C
:107F5000823048F58091AF019091B0012CDF603004
:107F600011F126D047DF1FC08038E9F421D080917D
:107F7000A5018093F100E8DE2BDF15C0882399F47A
:107F80009091AF01923078F49093A50111D020DF49
:107F90008091A501882321F48091E30091E087FD81
:107FA00094E09EBBEBDED9DE83FF089580E2FDDE28
:107FB00087EFCBCE8EB388230895FCDF69F08091E4
:107FC000E9008F931092E900C8DE83FF01C050DF03
:0A7FD0008F9187708093E9000895F7
:047FFC005DCEFBDC7F
:040000030000740085
:00000001FF
